:100000000C94C8010C94E5010C94E5010C94E501F5
:100010000C94E5010C94E5010C94E5010C94E501C8
:100020000C94E5010C94E5010C94E5010C94E501B8
:100030000C94E5010C94E5010C94E5010C94E501A8
:100040000C94E5010C94E5010C94E5010C94E50198
:100050000C94E5014572726F7220696E20676574B9
:1000600074696E6720636C757374657200456E64A5
:10007000206F6620436C75737465722043686169F4
:100080006E002046696C6520437265617465642169
:10009000002046696C6520617070656E646564213E
:1000A00000204E6F206672656520636C7573746501
:1000B00072210020456E7465722074657874202862
:1000C000656E642077697468207E293A00204E6F3F
:1000D000206672656520636C7573746572210020FB
:1000E0004372656174696E672046696C652E2E00E7
:1000F000202046696C6520616C72656164792065B9
:1001000078697374696E672C20617070656E6469BC
:100110006E6720646174612E2E0020467265652032
:100120004D656D6F72793A2000546F74616C204D8B
:10013000656D6F72793A20004572726F7220696E38
:100140002067657474696E6720636C75737465727B
:1001500000456E64206F6620436C75737465722071
:10016000436861696E002046696C65204372656171
:1001700074656421002046696C6520617070656E4D
:100180006465642100204E6F206672656520636C93
:100190007573746572210020456E746572207465F4
:1001A00078742028656E642077697468207E293A07
:1001B00000204E6F206672656520636C75737465F0
:1001C000722100204372656174696E672046696C14
:1001D000652E2E00202046696C6520616C72656179
:1001E0006479206578697374696E672C206170701A
:1001F000656E64696E6720646174612E2E00496EBD
:1002000076616C69642066696C654E616D652E2E41
:10021000004572726F7220696E2067657474696E32
:100220006720636C7573746572004572726F72201B
:10023000696E2067657474696E6720636C7573748A
:10024000657200524F4F5400444952002020200054
:1002500046494C45002020200046696C65206465B5
:100260006C65746564210044656C6574696E672E05
:100270002E0046696C6520646F6573206E6F742074
:1002800065786973742100534420696E697420662F
:1002900061696C2E2E0000407A10F35A00A0724E55
:1002A00018090010A5D4E80000E87648170000E41B
:1002B0000B54020000CA9A3B000000E1F505000063
:1002C00080969800000040420F000000A0860100C8
:1002D0000000102700000000E80300000000640098
:1002E000000000000A000000000001000000000003
:1002F0002C76D888DC674F0823DFC1DFAE59E1B127
:10030000B796E5E3E453C63AE651997696E8E6C235
:100310008426EB898C9B62ED407C6FFCEFBC9C9F3C
:1003200040F2BAA56FA5F490055A2AF75C936B6C5E
:10033000F9676DC11BFCE0E40D47FEF520E6B50052
:10034000D0ED902E0300943577050080841E0800C0
:1003500000204E0A000000C80C333333330F986E70
:1003600012831141EF8D2114893BE65516CFFEE62D
:10037000DB18D1844B381BF77C1D901DA4BBE424F3
:10038000203284725E228100C9F124ECA1E53D2770
:1003900011241FBECFE5D8E0DEBFCDBF13E0A0E63D
:1003A000B0E0ECEBFCE402C005900D92A235B10781
:1003B000D9F715E0A2E5B3E001C01D92A83CB10752
:1003C000E1F70E94D01C0C945C260C94000066237C
:1003D00011F0C09A01C0C098C198A29AA39AA49A99
:1003E000A59AAD98AC98AB98AA9887FDAD9A86FD72
:1003F000AC9A85FDAB9A84FDAA9AC29A00C0C298B5
:10040000AD98AC98AB98AA9883FDAD9A82FDAC9A52
:1004100081FDAB9A80FDAA9AC29A00C0C298AA9A9E
:10042000AB9AAC9AAD9A0895882311F0C09A01C096
:10043000C098C19AA298A398A498A598C29A00C0FF
:100440009A9B02C080E101C080E09B9980629C99E8
:1004500080649D998068C29800C0C29A00C09A9931
:1004600081609B9982609C9984609D998860C29804
:10047000089580E00E94140287FDFBCF84E090E0A5
:100480000197F1F780E00E94140208951F93182F3E
:100490000E943902812F60E00E94E7011F910895B8
:1004A0001F93182F0E943902812F61E00E94E701FB
:1004B0001F910895662311F4805809C0613011F42A
:1004C000805405C0623011F48C5601C08C520E94D9
:1004D000460208950E94390290E0089581E00E944A
:1004E0004602089582E00E94460208951F93182F45
:1004F0000E943902982F1A3099F4843110F480E464
:100500000BC08054843110F484E106C094519C32B5
:1005100010F080E001C084E580580E94460218C0B7
:10052000883011F480EC0BC0883411F484E907C0E2
:100530008C3111F484ED03C08C3521F480E860E047
:100540000E94E7010E943902812F61E00E94E701C9
:100550001F910895CF93DF93EC0102C00E947602B1
:1005600089918823D9F7DF91CF910895CF93DF93B5
:10057000EC0102C00E947602FE012196849188233C
:10058000C9F7DF91CF9108951F93182FB89AB99AA0
:10059000BA9AA29AA39AA49AA59A80E09DE7019795
:1005A000F1F7AB9AAA9AC29A00C0C29880E097E28B
:1005B0000197F1F7C29A00C0C29880E890E0FC0170
:1005C0003197F1F7C29A00C0C298FC013197F1F758
:1005D000AA98C29A00C0C2980197F1F788E20E94D7
:1005E000460288E00E9446020E946E0286E00E9457
:1005F0004602812F0E9446021F910895813049F0E2
:10060000813028F0823039F0833061F407C084EA09
:1006100003C084E801C084EC86BF04C084E986BFBF
:1006200080E0089506B607FEFDCF81B1887F08956A
:100630000F931F93142F00E0807F182B6770162BE9
:100640000F5F0333A9F080E00E94FE028833C1F3FC
:10065000883011F0803161F413B981E00E94FE020C
:10066000803271F3883361F3883111F480E001C086
:100670008FEF1F910F91089583E00E94FE0208956D
:1006800083B981E00E94FE02883211F480E008956F
:100690008FEF0895CF93DF93EC01662331F082E072
:1006A0000E94FE02803551F405C081E00E94FE02E6
:1006B000883521F483B1888380E001C08FEFDF911A
:1006C000CF9108958E9A88EE93E00197F1F78E9876
:1006D00080E58A95F1F780B38CEA93E00197F1F712
:1006E00080B390E026E0969587952A95E1F7817092
:1006F00008958E9A9DE09A95F1F7813009F48E98CD
:1007000085ED8A95F1F78E9808958E9A85E08A9501
:10071000F1F78E9888E28A95F1F780B390E036E0A1
:10072000969587953A95E1F78170089520E030E03D
:10073000482F50E07DE065EDCA01022E02C095957C
:1007400087950A94E2F78E9A972F9A95F1F780FD94
:100750008E98862F8A95F1F78E982F5F3F4F28301D
:10076000310551F788EC90E00197F1F7089540E0EA
:1007700020E030E0E5E058E261E070E08E9A8E2FF4
:100780008A95F1F78E98852F8A95F1F7869B08C098
:10079000CB01022E02C0880F991F0A94E2F7482B62
:1007A000852F8A95F1F72F5F3F4F2830310531F7BC
:1007B000842F089582E58DB91EB808958FB9779B6F
:1007C000FECF8FB108958FEF8FB9779BFECF8FB19A
:1007D0000895C19880648FB9779BFECF8FB1872F22
:1007E0009927AA27BB278FB9779BFECF8FB1CB0163
:1007F000AA27BB278FB9779BFECF8FB1BB27A72F27
:10080000962F852F8FB9779BFECF8FB14FB9779BEE
:10081000FECF8FB185E98FB9779BFECF8FB180E096
:100820002FEF02C0815031F02FB9779BFECF9FB1DF
:100830009F3FC1F38FEF8FB9779BFECF8FB1C19AE6
:10084000892F08950F931F93C19810E00FEF80E058
:100850000FB9779BFECF9FB18F5F8A30C9F780E0D9
:1008600040E050E060E070E00E94E9031F5F1F3F3E
:1008700059F4E7E8F2E004C05D9BFECF31968CB9F5
:1008800084918823C9F731C0813009F7C19A8FEF6D
:100890008FB9779BFECF8FB18FEF8FB9779BFECF4C
:1008A0008FB110E081E040E050E060E070E00E9435
:1008B000E90381E040E050E060E070E00E94E9037D
:1008C0001F5F1F3F91F0882369F78BE340E050E002
:1008D00060E070E00E94E90380E140E052E060E007
:1008E00070E00E94E90380E001C081E01F910F9158
:1008F0000895AF92BF92CF92DF92EF92FF920F9343
:100900001F937B018C0159016A01AB01BC0189E095
:10091000440F551F661F771F8A95D1F780E20E940A
:10092000E9038823F1F40894E108F10801091109A9
:10093000EA0CFB1C0C1D1D1DB9E0EE0CFF1C001F7A
:10094000111FBA95D1F781E2B801A7010E94E9030E
:10095000882339F486E240E050E060E070E00E94D5
:10096000E9031F910F91FF90EF90DF90CF90BF9020
:10097000AF900895AB01BC0199E0440F551F661F6D
:10098000771F9A95D1F781E10E94E903982F882378
:1009900091F5C19820E030E04FEF06C02150304083
:1009A00019F4C19A91E027C04FB9779BFECF8FB160
:1009B0008E3FA1F720E030E04FEF4FB9779BFECF9D
:1009C0008FB1F901E956FC4F80832F5F3F4F82E0E2
:1009D0002030380791F78FEF8FB9779BFECF8FB11B
:1009E0008FEF8FB9779BFECF8FB18FEF8FB9779B4A
:1009F000FECF8FB1C19A892F0895AB01BC0129E0C8
:100A0000440F551F661F771F2A95D1F788E10E9472
:100A1000E903882311F0982F55C0C1988EEF8FB944
:100A2000779BFECF8FB120E030E0F901E956FC4F13
:100A300080818FB9779BFECF8FB12F5F3F4F82E0D0
:100A40002030380791F78FEF8FB9779BFECF8FB1AA
:100A50008FEF8FB9779BFECF8FB18FEF8FB9779BD9
:100A6000FECF9FB1892F8F71853049F0C19A2AC07E
:100A70008FEF2F3F3807C9F02F5F3F4F03C020E0B3
:100A800030E09FEF9FB9779BFECF8FB1882381F332
:100A9000C19A8FEF8FB9779BFECF8FB1C1989FEF2F
:100AA00009C08FEF2F3F380719F4C19A91E00AC0AF
:100AB0002F5F3F4F9FB9779BFECF8FB1882389F37C
:100AC000C19A90E0892F08955F9BFECF8BB18CB1C6
:100AD00008955D9BFECF8CB90895DF93CF93CDB77A
:100AE000DEB72B970FB6F894DEBF0FBECDBF8130B7
:100AF00011F494E005C0823011F498E001C092E056
:100B0000DE011196E0E6F0E08BE001900D9281505D
:100B1000E1F79E012E5F3F4F842F8F70E92FF0E0A9
:100B20008A3020F4E20FF31F805D03C0E20FF31F51
:100B3000895C8083915019F4FE0131960CC0E4E089
:100B40007695679557954795EA95D1F7E5CF5D9BE3
:100B5000FECF31968CB980818823C9F72B960FB6CA
:100B6000F894DEBF0FBECDBFCF91DF910895FC0199
:100B700004C05D9BFECF31968CB984918823C9F760
:100B80000895FC0104C05D9BFECF31968CB9808135
:100B90008823C9F70895EF92FF920F931F93209136
:100BA000970530919805E0907903F0907A030091D1
:100BB0007B0310917C03625070408040904040E085
:100BC00050E00E94D8259B01AC012E0D3F1D401F17
:100BD000511FB901CA011F910F91FF90EF90089525
:100BE0004F925F926F927F928F929F92AF92BF923D
:100BF000CF92DF92EF92FF920F931F93CF93DF93E9
:100C00005B016C01842E280139018091B50590911A
:100C1000B605F2E0AA0CBB1CCC1CDD1CFA95D1F782
:100C200020918103309182037C0100E010E08091EB
:100C3000AD059091AE05A091AF05B091B005E80E5D
:100C4000F91E0A1F1B1F40E050E0C601B5010E94BB
:100C50000326E20EF31E041F151FC0918103D091DD
:100C600082039924C801B7010E94BA04882321F0A5
:100C700093948AE09816B1F79E0140E050E0C601D7
:100C8000B5010E940326FB01E956FC4F882031F490
:100C900020813181428153815F700CC0408251823A
:100CA00062827382C801B7010E94FD0420E030E037
:100CB00040E050E0B901CA01DF91CF911F910F913F
:100CC000FF90EF90DF90CF90BF90AF909F908F906C
:100CD0007F906F905F904F900895CF92DF92EF9248
:100CE000FF920F931F93D82EC62E79018A0160912F
:100CF000AD057091AE058091AF059091B0056F5F25
:100D00007F4F8F4F9F4F0E94BA048091970390911D
:100D10009803A0919903B0919A0382559245A146F8
:100D2000B14409F054C080917B0590917C05A0915D
:100D30007D05B0917E0582579247A144B14609F0E6
:100D400046C08091930590919405A0919505B0912E
:100D5000960580509040A545BA4AC9F5CC20A9F423
:100D600081E0D81649F420917F05309180054091AB
:100D70008105509182052FC0209183053091840513
:100D8000409185055091860526C021E0D21649F490
:100D9000E0927F05F0928005009381051093820513
:100DA00008C0E0928305F0928405009385051093B6
:100DB00086056091AD057091AE058091AF0590916B
:100DC000B0056F5F7F4F8F4F9F4F0E94FD042FEF45
:100DD0003FEF4FEF5FEFB901CA011F910F91FF90F5
:100DE000EF90DF90CF9008956F927F928F929F92B5
:100DF000AF92BF92CF92DF92EF92FF920F931F9329
:100E00001092AD051092AE051092AF051092B0058C
:100E100060E070E080E090E00E94BA048091970367
:100E2000893E19F18B3E09F18091950590919605C7
:100E300085559A4A09F0B0C060915D0570915E05D4
:100E400080915F05909160056093AD057093AE054C
:100E50008093AF059093B0050E94BA0480919703E8
:100E6000893E19F08B3E09F097C08091A2039091C2
:100E7000A30390938203809381038091A40390E065
:100E80009093980580939705A090A503B090A60332
:100E9000B092B605A092B5058091C3039091C403AA
:100EA000A091C503B091C60380938F0390939003E4
:100EB000A0939103B0939203E090B505F090B6052E
:100EC0006091A70370E080E090E02091BB03309137
:100ED000BC034091BD035091BE030E94D8253B0145
:100EE0004C0100E010E08091B3039091B403A09115
:100EF000B503B091B603E80EF91E0A1F1B1FE60CDE
:100F0000F71C081D191DE0927903F0927A030093F3
:100F10007B0310937C032091970530919805CC2496
:100F2000DD246091B7037091B8038091B90390916B
:100F3000BA036A197B098C099D0966197709880922
:100F4000990940E050E00E940326C901DA0180932C
:100F5000830390938403A0938503B093860381E079
:100F600060E020E030E040E050E00E946D0620911B
:100F700083033091840340918503509186032617A3
:100F800037074807590718F41092C30503C081E0DA
:100F90008093C30580E001C081E01F910F91FF9015
:100FA000EF90DF90CF90BF90AF909F908F907F9009
:100FB0006F9008950F931F93DF93CF93CDB7DEB754
:100FC0002B970FB6F894DEBF0FBECDBF8C01582F04
:100FD000A12FFC0140E080818E3219F4493030F0BD
:100FE00013C04F5F31964C30B1F70EC0BE016F5F3A
:100FF0007F4F852F9A2F9C01F901DB010EC05D9B6D
:10100000FECF31968CB902C0EEEFF1E084918823D7
:10101000B1F781E052C081918D938E2F851B84178B
:10102000D0F3842F9E012F5F3F4F90E205C0F9015E
:10103000E80FF11D90838F5F8830C9F7242F2F5F51
:10104000AE014F5F5F4F30E2F801E20FF11D90817A
:10105000992359F0FA01E80FF11D90832F5F07C023
:10106000FA01E80FF11D30838F5F8B30C8F38F5F7B
:101070008B3050F39E01245F3F4FFB019081892FFD
:1010800081568A3110F4905290836F5F7F4F6217C0
:10109000730799F720E030E0AE014F5F5F4FF80132
:1010A000E20FF31FDA01A20FB31F8C9180832F5F31
:1010B0003F4F2B30310599F780E02B960FB6F8940F
:1010C000DEBF0FBECDBFCF91DF911F910F9108956D
:1010D0006F927F928F929F92AF92BF92CF92DF9248
:1010E000EF92FF920F931F9360783B014C01B2E0A7
:1010F000660C771C881C991CBA95D1F75B016C01B2
:1011000050C0E090B505F090B60520918103309174
:10111000820300E010E08091AD059091AE05A091B2
:10112000AF05B091B005E80EF91E0A1F1B1F40E085
:1011300050E0C401B3010E940326E20EF31E041F17
:10114000151FC801B7010E94BA0460E0E62FF0E065
:10115000EE0FFF1FEE0FFF1FE956FC4F80819181BC
:10116000A281B381BF700097A105B10539F4A60132
:101170009501260F311D411D511D25C06F5F60383F
:1011800029F780E890E0A0E0B0E0A80EB91ECA1EE2
:10119000DB1E80E092E0A0E0B0E0680E791E8A1EBF
:1011A0009B1E8091830390918403A0918503B0914D
:1011B0008603A816B906CA06DB0608F4A2CF20E00B
:1011C00030E040E050E0B901CA011F910F91FF905B
:1011D000EF90DF90CF90BF90AF909F908F907F90D7
:1011E0006F9008959F92AF92BF92CF92DF92EF924D
:1011F000FF920F93DF93CF93CDB7DEB763970FB610
:10120000F894DEBF0FBECDBF6B017C01DE011196ED
:10121000EBE6F0E083E101900D928150E1F70CE004
:101220008CE2982E053011F0093029F4FE01E00F10
:10123000F11D908201505E01A00EB11CC701B601E4
:101240002AE030E040E050E00E9403266063F501B0
:101250006083C701B6012AE030E040E050E00E9420
:101260000326C901DA016C017D01C114D104E10436
:10127000F10419F4FE01319607C0015099F6FACF36
:101280005D9BFECF31968CB980818823C9F7639628
:101290000FB6F894DEBF0FBECDBFCF91DF910F9197
:1012A000FF90EF90DF90CF90BF90AF909F90089508
:1012B0002F923F924F925F926F927F928F929F9266
:1012C000AF92BF92CF92DF92EF92FF920F931F9354
:1012D000A0908303B0908403C0908503D0908603D0
:1012E0006091970570919805209181033091820358
:1012F0005D9BFECF8DE08CB95D9BFECF8AE08CB903
:101300005D9BFECF8DE08CB95D9BFECF8AE08CB9F2
:10131000E9E2F1E004C05D9BFECF31968CB9849187
:101320008823C9F780E090E040E050E00E94D82593
:10133000A60195010E94D8250E94F20881E060E094
:1013400020E030E040E050E00E946D061B012C01DF
:101350008091830390918403A0918503B0918603CB
:1013600082159305A405B50508F07CC01092C3054D
:10137000A0908F03B0909003C0909103D0909203FF
:1013800072E0AA0CBB1CCC1CDD1C7A95D1F7222480
:1013900033242101662477244301E090B505F090C1
:1013A000B605209181033091820300E010E0809126
:1013B000AD059091AE05A091AF05B091B005E80ED6
:1013C000F91E0A1F1B1F40E050E0C601B5010E9434
:1013D0000326E20EF31E041F151FC801B7010E9469
:1013E000BA04A401930160E070E0FB01E956FC4FF0
:1013F00080819181A281B381BF700097A105B10561
:1014000029F40894211C311C411C511C2F5F3F4FB3
:101410004F4F5F4F8091830390918403A091850388
:10142000B09186030296A11DB11D281739074A07FE
:101430005B07C1F0C901861997096C5F7F4F02E015
:101440006030700791F6E12C62E0F62E012D112D2F
:10145000AE0CBF1CC01ED11E8038910518F039019A
:101460004A019BCF8091C305882331F481E061E07C
:10147000A20191010E946D0681E08093C305209135
:1014800097053091980560918103709182035D9B6F
:10149000FECF8DE08CB95D9BFECF8AE08CB9EAE18E
:1014A000F1E004C05D9BFECF31968CB98491882316
:1014B000C9F780E090E040E050E00E94D825A2010A
:1014C00091010E94D8250E94F2085D9BFECF8DE01D
:1014D0008CB95D9BFECF8AE08CB91F910F91FF9074
:1014E000EF90DF90CF90BF90AF909F908F907F90C4
:1014F0006F905F904F903F902F900895DF92EF9202
:10150000FF920F931F93D82EDB01CA01F9E0B69525
:10151000A79597958795FA95D1F75170607070707F
:10152000411551056105710519F4AC01BD0106C0F5
:10153000AC01BD014F5F5F4F6F4F7F4FDB01CA01B1
:10154000E3E0B695A79597958795EA95D1F747700B
:10155000507060707070411551056105710519F486
:101560007C018D0107C07C018D010894E11CF11CF8
:10157000011D111D8091C3058823D9F081E060E031
:1015800020E030E040E050E00E946D06DD2039F4BC
:101590009B01AC012E0D3F1D401F511F06C09B013A
:1015A000AC012E193F09400B510B81E061E00E9414
:1015B0006D061F910F91FF90EF90DF9008952F928D
:1015C0003F924F925F926F927F928F929F92AF92D3
:1015D000BF92CF92DF92EF92FF920F931F93DF9310
:1015E000CF93CDB7DEB728970FB6F894DEBF0FBE06
:1015F000CDBF382E7E836D83A0908F03B090900373
:10160000C0909103D0909203282E2A9420919705A0
:1016100030919805E0907903F0907A0300917B0374
:1016200010917C03C601B50162507040804090402B
:1016300040E050E00E94D8253B014C016E0C7F1C1D
:10164000801E911EEE24FF2487018FC1D801C7019F
:10165000860D971DA81DB91D89839A83AB83BC8312
:10166000BC01CD010E94BA0480E2482E512C6DC10C
:10167000DA01A956BC4FB887AF83F201E956FC4F97
:10168000B0978081B096882381F43A94B1E0B31585
:1016900008F49BC1E2E7F2E004C05D9BFECF319607
:1016A0008CB984918823C9F790C1853E09F449C15A
:1016B000759790819F3009F444C1E1E0E21508F488
:1016C000ECC020E030E08F819885820F931FAD81C0
:1016D000BE81A20FB31FFC0190818C91981709F075
:1016E00030C1822F8F5F2F5F3F4F2B30310559F76D
:1016F0008B3009F026C1F1E03F1609F041C0898125
:101700009A81AB81BC818093C4059093C505A09359
:10171000C605B093C705CA01A0E0B0E08093680396
:1017200090936903A0936A03B0936B03AF81B8856C
:1017300054968D919C915597A0E0B0E0DC019927DB
:101740008827EF81F885228D338D40E050E0822B91
:10175000932BA42BB52B8093B7059093B805A0933A
:10176000B905B093BA05848D958DA68DB78D8093FC
:101770007D0390937E03A0937F03B093800327C1E2
:101780005D9BFECF8DE08CB95D9BFECF8AE08CB96E
:10179000E7E6F2E004C05D9BFECF31968CB9849100
:1017A0008823C9F75D9BFECF8DE08CB95D9BFECF92
:1017B0008AE08CB95D9BFECF8DE08CB95D9BFECF3E
:1017C0008AE08CB9AF81B88554968D919C915597DC
:1017D000A0E0B0E05C0199248824EF81F885828D37
:1017E000938DA0E0B0E0882A992AAA2ABB2A85EE28
:1017F000808369817A818B819C810E94FD04AF8105
:10180000B8855C964D915D916D917C915F9780E07C
:101810000E947E0A82E060E020E030E040E050E09C
:101820000E946D0686169706A806B90630F482E077
:1018300061E0A50194010E946D06C501B40140E07C
:1018400000E010E020E030E00E94F005F62EE72EE8
:10185000D82EC92EC501B40141E000E010E020E01F
:1018600030E00E94F0058F2D9E2DAD2DBC2D4C013A
:101870005D01B7EF8B16BFEF9B06BFEFAB06BFE076
:10188000BB06D8F2E9E5F2E004C05D9BFECF3196DD
:101890008CB984918823C9F798C05D9BFECFEDE099
:1018A000ECB95D9BFECFFAE0FCB980E006C0883061
:1018B00021F45D9BFECF20E22CB9EF81F885E80F83
:1018C000F11DE0815D9BFECFECB98F5F8B3078F32B
:1018D000E5E5F2E004C05D9BFECF31968CB98491C2
:1018E0008823C9F7903119F1983019F4E3E4F2E054
:1018F00025C0E0E5F2E004C05D9BFECF31968CB9D7
:1019000084918823C9F7ECE4F2E004C05D9BFECF2C
:1019100031968CB984918823C9F7F201ED56FC4FBA
:1019200060817181828193810E94F2080AC0E8E49B
:10193000F2E004C05D9BFECF31968CB98491882380
:10194000C9F780E290E0480E591EA2014052504073
:1019500080918103909182034817590708F488CE3B
:101960000894E11CF11C011D111D809197059091B7
:101970009805A0E0B0E0E816F9060A071B0708F48E
:1019800065CEC601B50140E000E010E020E030E0A7
:101990000E94F0055B016C0197EFA9169FEFB90655
:1019A0009FEFC9069FE0D90680F4A114B104C104D9
:1019B000D10409F02BCEEAE2F2E004C05D9BFECF39
:1019C00031968CB984918823C9F718861F828F813C
:1019D000988528960FB6F894DEBF0FBECDBFCF9185
:1019E000DF911F910F91FF90EF90DF90CF90BF900C
:1019F000AF909F908F907F906F905F904F903F90AF
:101A00002F900895CF93DF93EC010E94DA0788238B
:101A100021F482E0BE010E94DF0ADF91CF91089598
:101A20002F923F924F925F926F927F928F929F92EE
:101A3000AF92BF92CF92DF92EF92FF920F931F93DC
:101A4000DF93CF9300D000D0CDB7DEB7E82E8B0167
:101A5000CB010E94DA07882311F082E0A7C081E061
:101A6000B8010E94DF0A009709F49FC021E0E21646
:101A700011F481E09BC0DC0154962D913C91559767
:101A80005A964D915C915B975C968D919D910D90CE
:101A9000BC91A02D89839A83AB83BC835D9BFECFD1
:101AA0008DE08CB95D9BFECF8AE08CB95D9BFECF4B
:101AB0008DE08CB95D9BFECFC901A0E0B0E06C0168
:101AC000BB24AA24CA01A0E0B0E0A82AB92ACA2AE5
:101AD000DB2A8AE08CB92224332421012091970546
:101AE00030919805E0907903F0907A0300917B03A0
:101AF00010917C03C601B501625070408040904057
:101B000040E050E00E94D8253B014C016E0C7F1C48
:101B1000801E911E10E025C0C401B301610F711D2C
:101B2000811D911D0E94BA0480E090E0FC01E956FD
:101B3000FC4FE0815D9BFECFECB929813A814B815E
:101B40005C81221633064406550678F50894211C5C
:101B5000311C411C511C019632E08030930731F753
:101B60001F5F2091970530919805812F90E0821793
:101B7000930790F2C601B50140E000E010E020E0DC
:101B800030E00E94F0055B016C0161157105810573
:101B9000910509F0A3CFE1E1F2E004C05D9BFECF27
:101BA00031968CB984918823C9F780E00F900F900B
:101BB0000F900F90CF91DF911F910F91FF90EF90B9
:101BC000DF90CF90BF90AF909F908F907F906F905D
:101BD0005F904F903F902F9008952F923F924F9299
:101BE0005F926F927F928F929F92AF92BF92CF92AD
:101BF000DF92EF92FF920F931F93DF93CF93CDB7B6
:101C0000DEB727970FB6F894DEBF0FBECDBF9F8318
:101C10008E8381E06E817F810E94100D813009F0FA
:101C20005CC0E4EDF1E004C05D9BFECF31968CB961
:101C300084918823C9F76090B7057090B8058090AB
:101C4000B9059090BA05AA24BB246501C401B3016B
:101C500040E000E010E020E030E00E94F0056F3F3F
:101C60002FEF72072FEF82072FE0920741F00894C1
:101C7000A11CB11CC11CD11C3B014C01E7CF209120
:101C80009705309198056091810370918203E090EF
:101C90008103F090820380E090E040E050E00E94F9
:101CA000D825A60195010E94D8259B01AC01609121
:101CB0007D0370917E0380917F0390918003621B6E
:101CC000730B840B950B00E010E0A80197010E94B4
:101CD0000326A22E21E02D836AC0823009F440C37E
:101CE0005D9BFECF8DE08CB95D9BFECF8AE08CB909
:101CF000E3ECF1E004C05D9BFECF31968CB984919A
:101D00008823C9F782E060E020E030E040E050E066
:101D10000E946D069B01AC01809183039091840326
:101D2000A0918503B091860382179307A407B50796
:101D300040F420918F033091900340919103509192
:101D40009203CA01B9010E9468083B014C01611568
:101D500071058105910599F45D9BFECF8DE08CB9ED
:101D60005D9BFECF8AE08CB9E1EBF1E004C05D9BA6
:101D7000FECF31968CB984918823C9F7F1C241E036
:101D80000FEF1FEF2FEF3FE00E94F005C401AA27DD
:101D9000BB279C838B837A82698210927D03109289
:101DA0007E0310927F031092800320E01D822A2C74
:101DB0003324442455243AE0B32EC401B3016250C5
:101DC0007040804090402223E1F1209197053091AE
:101DD0009805E0907903F0907A0300917B031091CD
:101DE0007C03E20CF31C041D151D40E050E00E9432
:101DF000D825E60EF71E081F191FE0929303F092F4
:101E0000940300939503109396036091930370914C
:101E1000940380919503909196030E94BA042091B7
:101E200081033091820340E050E060917D03709126
:101E30007E0380917F03909180030E9403260A2DE8
:101E40001FC02091970530919805E0907903F0909C
:101E50007A0300917B0310917C0340E050E00E94E4
:101E6000D825E60EF71E081F191FE0929303F09283
:101E70009403009395031093960300E060E070E0F4
:101E80005D9BFECF8DE08CB95D9BFECFBCB8E7E9D2
:101E9000F1E004C05D9BFECF31968CB9849188231C
:101EA000C9F75F9BFECF8BB11CB1183029F56115C6
:101EB0007105B9F35D9BFECF98E09CB95D9BFECFA9
:101EC000A0E2ACB95D9BFECFB8E0BCB961507040F8
:101ED00080917D0390917E03A0917F03B091800358
:101EE0000197A109B10980937D0390937E03A0938C
:101EF0007F03B0938003D5CF5D9BFECF1CB9FB0160
:101F0000E956FC4F10836F5F7F4F80917D03909166
:101F10007E03A0917F03B09180030196A11DB11DA6
:101F200080937D0390937E03A0937F03B0938003FF
:101F30001D30A1F45D9BFECFBCB8FB01E956FC4F00
:101F4000B0826F5F7F4F0196A11DB11D80937D030D
:101F500090937E03A0937F03B0938003E2E0603010
:101F60007E0749F5609193037091940380919503E6
:101F7000909196030E94FD040F5F20919705309188
:101F80009805802F90E082179307C9F08091930302
:101F900090919403A0919503B09196030196A11D91
:101FA000B11D8093930390939403A0939503B093F2
:101FB000960360E070E01E3709F073CF04C01E374F
:101FC000B9F560E070E080917D0390917E03A0916F
:101FD0007F03B09180030197A109B10980937D032C
:101FE00090937E03A0937F03B09380036150704071
:101FF00006C0FB01E956FC4F10826F5F7F4FF2E095
:1020000060307F07B0F360919303709194038091E7
:102010009503909196030E94FD0482E061E0A40183
:1020200093010E946D062D81222309F483C032C0E2
:10203000C401B3010E9468086B017C016115710540
:102040008105910599F45D9BFECF8DE08CB95D9B78
:10205000FECF8AE08CB9E5E8F1E004C05D9BFECFDD
:1020600031968CB984918823C9F77AC1C401B30130
:1020700041E0970186010E94F005C701B60141E0E9
:102080000FEF1FEF2FEF3FE00E94F00520E0360139
:10209000470193CE6091C4057091C5058091C60536
:1020A0009091C7050E94BA04E0916803F09169031A
:1020B000E956FC4F20917D0330917E0340917F03D0
:1020C00050918003848D958DA68DB78D79018A01FD
:1020D000E81AF90A0A0B1B0B248F358F468F578F8E
:1020E0006091C4057091C5058091C6059091C705A2
:1020F0000E94FD0481E0B801A7010E947E0A5D9B59
:10210000FECF8DE08CB95D9BFECF8AE08CB9E5E710
:10211000F1E004C05D9BFECF31968CB98491882399
:10212000C9F75D9BFECF8DE08CB95D9BFECF8AE049
:102130008CB916C180908F0390909003A09091036A
:10214000B090920322242091970530919805E09059
:102150007903F0907A0300917B0310917C03C50111
:10216000B401625070408040904040E050E00E94D6
:10217000D8252B013C014E0C5F1C601E711E3324C0
:1021800094C073016201C30CD11CE11CF11CC70196
:10219000B6010E94BA0400E210E07CC0AF014956CB
:1021A0005C4F222019F0DA011C92DAC0F801E958DC
:1021B000FC4FE081EE2319F0E53E09F069C020E014
:1021C00030E0BA01620F731FAE81BF81A20FB31F4F
:1021D0008C91FB0180832F5F3F4F2B30310589F7B6
:1021E000F801E956FC4F759720E221931192119264
:1021F00084E896E981939193A7E3BAE3A193B1931D
:10220000B183A083349681939193B183A083349753
:102210008B819C81918380833696A981BA81A19319
:10222000B19380917D0390917E03A0917F03B09143
:10223000800380839183A283B383C701B6010E9488
:10224000FD045D9BFECFBDE0BCB95D9BFECFEAE027
:10225000ECB95D9BFECFFDE0FCB95D9BFECF2AE0B3
:102260002CB9E6E6F1E004C05D9BFECF31968CB957
:1022700084918823C9F740917D0350917E0360913A
:102280007F037091800381E00E947E0A22242394C0
:10229000005E1F4F8091810390918203F801B097F7
:1022A000E817F90708F47ACF339420919705309115
:1022B0009805832D90E08217930708F462CFC5013B
:1022C000B40140E000E010E020E030E00E94F005C2
:1022D0006B017C0187EFC8168FEFD8068FEFE806F9
:1022E0008FE0F80658F19FEFC9169FEFD9069FEFD0
:1022F000E9069FE0F90619F0E1E5F1E01BC0C50130
:10230000B4010E9468086B017C01C501B40141E081
:10231000970186010E94F005C701B60141E00FEF69
:102320001FEF2FEF3FE00E94F00508C05D9BFECF3E
:1023300031968CB984918823C9F712C046015701A0
:10234000C114D104E104F10409F0FDCEE8E3F1E0A9
:1023500004C05D9BFECF31968CB984918823C9F768
:1023600027960FB6F894DEBF0FBECDBFCF91DF9199
:102370001F910F91FF90EF90DF90CF90BF90AF90A3
:102380009F908F907F906F905F904F903F902F9095
:1023900008952F923F924F925F926F927F928F9209
:1023A0009F92AF92BF92CF92DF92EF92FF920F93E4
:1023B0001F93DF93CF93CDB7DEB72B970FB6F8946B
:1023C000DEBF0FBECDBF9987888781E0688579859C
:1023D0000E94100D813009F05CC0E0EFF0E004C015
:1023E0005D9BFECF31968CB984918823C9F76090AC
:1023F000B7057090B8058090B9059090BA05AA24E9
:10240000BB246501C401B30140E000E010E020E01E
:1024100030E00E94F0056F3F2FEF72072FEF820729
:102420002FE0920741F00894A11CB11CC11CD11CE3
:102430003B014C01E7CF20919705309198056091C1
:10244000810370918203E0908103F090820380E029
:1024500090E040E050E00E94D825A60195010E943E
:10246000D8259B01AC0160917D0370917E03809122
:102470007F0390918003621B730B840B950B00E02C
:1024800010E0A80197010E9403262D8321E02E83EE
:102490006AC0823009F423C35D9BFECF8DE08CB906
:1024A0005D9BFECF8AE08CB9EFEDF0E004C05D9B50
:1024B000FECF31968CB984918823C9F782E060E021
:1024C00020E030E040E050E00E946D069B01AC014E
:1024D0008091830390918403A0918503B09186033A
:1024E00082179307A407B50740F420918F0330911A
:1024F00090034091910350919203CA01B9010E9447
:1025000068083B014C01611571058105910599F43D
:102510005D9BFECF8DE08CB95D9BFECF8AE08CB9D0
:10252000EDECF0E004C05D9BFECF31968CB9849158
:102530008823C9F7D4C241E00FEF1FEF2FEF3FE030
:102540000E94F005C401AA27BB279C838B837A8253
:10255000698210927D0310927E0310927F03109285
:10256000800320E01E82AA24BB248D81282E3324E0
:1025700044245524C401B30162507040804090400F
:102580002223E1F12091970530919805E09079039D
:10259000F0907A0300917B0310917C03E20CF31C12
:1025A000041D151D40E050E00E94D825E60EF71EE0
:1025B000081F191FE0929303F09294030093950370
:1025C0001093960360919303709194038091950307
:1025D000909196030E94BA04209181033091820366
:1025E00040E050E060917D0370917E0380917F0315
:1025F000909180030E9403260D811FC020919705B2
:1026000030919805E0907903F0907A0300917B0374
:1026100010917C0340E050E00E94D825E60EF71EA2
:10262000081F191FE0929303F092940300939503FF
:102630001093960300E060E070E05D9BFECF9DE0AC
:102640009CB95D9BFECFAAE0ACB9E3EBF0E004C01F
:102650005D9BFECF31968CB984918823C9F7E2E562
:10266000EE2EE3E0FE2EEA0CFB1CB6E1AB16B10445
:1026700010F010E005C0F7011081112309F41EE7E6
:102680000894A11CB11C5D9BFECF1CB9FB01E9564F
:10269000FC4F10836F5F7F4F80917D0390917E038D
:1026A000A0917F03B09180030196A11DB11D80937D
:1026B0007D0390937E03A0937F03B0938003F2E0A9
:1026C00060307F0749F56091930370919403809186
:1026D0009503909196030E94FD040F5F209197054A
:1026E00030919805802F90E082179307E1F0809158
:1026F000930390919403A0919503B0919603019652
:10270000A11DB11D8093930390939403A09395030F
:10271000B093960360E070E00894E11CF11C1E3752
:1027200009F0A3CF04C01E37B9F560E070E08091D6
:102730007D0390917E03A0917F03B0918003019768
:10274000A109B10980937D0390937E03A0937F0339
:10275000B09380036150704006C0FB01E956FC4F06
:1027600010826F5F7F4F22E060307207B0F360919C
:1027700093037091940380919503909196030E9426
:10278000FD0482E061E0A40193010E946D068E8148
:10279000882309F483C032C0C401B3010E946808D1
:1027A0006B017C01611571058105910599F45D9BB3
:1027B000FECF8DE08CB95D9BFECF8AE08CB9E1EA5B
:1027C000F0E004C05D9BFECF31968CB984918823E4
:1027D000C9F785C1C401B30141E0970186010E9498
:1027E000F005C701B60141E00FEF1FEF2FEF3FE00B
:1027F0000E94F00520E036014701BCCE6091C4057F
:102800007091C5058091C6059091C7050E94BA04D4
:10281000E0916803F0916903E956FC4F20917D0334
:1028200030917E0340917F0350918003848D958D7C
:10283000A68DB78D79018A01E81AF90A0A0B1B0BDC
:10284000248F358F468F578F6091C4057091C505D1
:102850008091C6059091C7050E94FD0481E0B801F2
:10286000A7010E947E0A5D9BFECF8DE08CB95D9B27
:10287000FECF8AE08CB9E1E9F0E004C05D9BFECFB9
:1028800031968CB984918823C9F75D9BFECF8DE08A
:102890008CB95D9BFECF8AE08CB921C180908F03FB
:1028A00090909003A0909103B09092031F8257E301
:1028B000252E5AE3352E2091970530919805E0900A
:1028C0007903F0907A0300917B0310917C03C5019A
:1028D000B401625070408040904040E050E00E945F
:1028E000D8252B013C014E0C5F1C601E711EDD249F
:1028F0009BC083017201ED0CF11C011D111DC8016B
:10290000B7010E94BA04A0E2B0E0BB87AA8780C0EA
:10291000AF0149565C4FBF81BB2319F0FA01108209
:10292000DEC0EA85FB85E958FC4FE081EE2319F013
:10293000E53E09F068C020E030E0BA01620F731F85
:10294000A885B985A20FB31F8C91DB018C932F5FF3
:102950003F4F2B30310589F7EA85FB85E956FC4F5F
:102960007597B0E2B1931192119284E896E9819340
:102970009193219231923182208234968193919366
:10298000318220823497AB81BC81B183A08336969B
:1029900089819A818193919380917D0390917E03A7
:1029A000A0917F03B091800380839183A283B3833E
:1029B000C801B7010E94FD045D9BFECF9DE09CB95C
:1029C0005D9BFECFAAE0ACB95D9BFECFBDE0BCB97C
:1029D0005D9BFECFEAE0ECB9E2E8F0E004C05D9B6D
:1029E000FECF31968CB984918823C9F740917D033D
:1029F00050917E0360917F037091800381E00E947B
:102A00007E0AF1E0FF838A859B8580969B878A8773
:102A10008091810390918203EA85FB85B097E81746
:102A2000F90708F475CFD394209197053091980554
:102A30008D2D90E08217930708F45BCFC501B40198
:102A400040E000E010E020E030E00E94F0056B0183
:102A50007C0197EFC9169FEFD9069FEFE9069FE02B
:102A6000F90658F1AFEFCA16AFEFDA06AFEFEA0694
:102A7000AFE0FA0619F0EDE6F0E01BC0C501B401C5
:102A80000E9468086B017C01C501B40141E0970117
:102A900086010E94F005C701B60141E00FEF1FEF6C
:102AA0002FEF3FE00E94F00508C05D9BFECF3196FE
:102AB0008CB984918823C9F712C046015701C1140B
:102AC000D104E104F10409F0F6CEE4E5F0E004C03D
:102AD0005D9BFECF31968CB984918823C9F72B96E4
:102AE0000FB6F894DEBF0FBECDBFCF91DF911F911F
:102AF0000F91FF90EF90DF90CF90BF90AF909F909D
:102B00008F907F906F905F904F903F902F9008959F
:102B1000482F6AE00E94F725282F30E0A4E0220F1A
:102B2000331FAA95E1F7842F0E94F725892F820F82
:102B30000895282F22952F709AE0299F9001112443
:102B40008F70820F08951F93CF93DF93AF9A809178
:102B5000BB058F778093BB0580ED90E060E070E06F
:102B600040E00E94180380E00E944003CBEBD5E0D8
:102B700010E0123031F48091BD050E9488158F7BE2
:102B800003C088810E9488150E9440031F5F219620
:102B9000173079F70E943C03AF98DF91CF911F91D6
:102BA0000895833091F0843038F4813009F4ADC059
:102BB000823009F0D5C022C0853071F0853008F42C
:102BC00040C0863009F0CCC084C040E050E0E8E767
:102BD000F5E068EA76E17AC021E030E048EE53E0C3
:102BE000949ACA010197F1F79498CA010197F1F7F5
:102BF0002F5F3F4F2C33310599F7089521E030E0E6
:102C00004CED55E0949ACA010197F1F79498CA01E6
:102C10000197F1F72F5F3F4F2C33310599F721E0F2
:102C200030E044EF51E0949ACA010197F1F794988B
:102C3000CA010197F1F72F5F3F4F243B310599F708
:102C4000089521E030E044EF51E0949ACA010197E1
:102C5000F1F79498CA010197F1F72F5F3F4F243B9A
:102C6000310599F721E030E04CED55E0949ACA0126
:102C70000197F1F79498CA010197F1F72F5F3F4F41
:102C80002C33310599F70895949ACF010197F1F704
:102C90009498CF010197F1F72F5F3F4F213931050C
:102CA00099F721E030E0949ACB010197F1F79498DD
:102CB000CB010197F1F72F5F3F4F2332310599F791
:102CC0004F5F5F4F4230510509F44AC021E030E0C8
:102CD000DBCF21E030E04CED55E0949ACA0101973A
:102CE000F1F79498CA010197F1F72F5F3F4F81E008
:102CF0002E35380791F78CED95E028EC30E0F9019E
:102D00003197F1F70197D9F7089521E030E048E7CE
:102D100055E0949ACA010197F1F79498CA01019776
:102D2000F1F72F5F3F4F2233310599F78CED95E096
:102D300028EC30E0F9013197F1F70197D9F721E05C
:102D400030E048E755E0949ACA010197F1F794986A
:102D5000CA010197F1F72F5F3F4F2233310599F7F1
:102D60000895DB9ADC9890E5892F8A95F1F7CA9946
:102D700003C021E030E024C0C99903C022E030E064
:102D80001FC0C89903C023E030E01AC0DC9ADB986A
:102D9000892F8A95F1F7CA9903C024E030E010C06A
:102DA000C99903C025E030E00BC0C89903C026E0F4
:102DB00030E006C0DB9A892F8A95F1F720E030E0F9
:102DC000C90108950E94B11618161906DCF380E9AE
:102DD00091E028EC30E0F9013197F1F70197D9F74C
:102DE00008950E946E028EE790E00E94AA0288EE8B
:102DF00093E028EC30E0F9013197F1F70197D9F72A
:102E00000E94A3150E946E028DE890E00E94AA0223
:102E100082E00E94D11508958C9A80E58A95F1F799
:102E200081E00E94D115A69AA79AD49AD39ADC9AE7
:102E3000DB9AD298D198D098DA9AD99AD89AF894FD
:102E40008FEE88BB8FEB87BB82E58DB91EB815BEB0
:102E50001BBE19BE84EF91E028EC30E0F9013197F8
:102E6000F1F70197D9F71AB81BB886E880BD89E158
:102E700089B910BC88E18AB98CE00E94C4020E9422
:102E80006E020895FF920F931F93DF93CF930F92DB
:102E9000CDB7DEB7AF9A80ED90E060E070E040E043
:102EA0000E94180380E00E9440030E943C0380EDD2
:102EB00090E060E070E041E00E9418038E010F5F37
:102EC0001F4FC80161E00E944A032981822F8F773A
:102ED00082958F709AE0F92E8F9DC00111242F707A
:102EE000280F2093BB05C80161E00E944A03298195
:102EF000822F82958F708F9DC00111242F70280F13
:102F00002093BC05C80161E00E944A038981282FF3
:102F10002F7086FF02C08F7101C08F7382958F70F2
:102F20008F9DC0011124280F2093BD058E010F5FD6
:102F30001F4FC80161E00E944A032981822F8295B8
:102F40008F70BAE0FB2E8F9DC00111242F70280FC7
:102F50002093BE05C80161E00E944A032981822FA7
:102F600082958F708F9DC00111242F70280F2093A0
:102F7000BF05C80161E00E944A032981822F829522
:102F80008F708F9DC00111242F70280F2093C005D2
:102F9000C80160E00E944A032981822F82958F70C8
:102FA0008F9DC00111242F70280F2093C1050E940E
:102FB0003C03AF982CE633E0D9011D929D01B3E0AC
:102FC00029373B07C9F7EDB7FEB73A970FB6F89424
:102FD000FEBF0FBEEDBF31962D503040ADB7BEB72E
:102FE00012963C932E93119789E990E09383828304
:102FF0008091C105848315828091C00586831782E4
:103000008091BF05808711860E94FD20EDB7FEB735
:103010003A960FB6F894FEBF0FBEEDBF0F90CF915A
:10302000DF911F910F91FF900895AF9A0E946E0259
:103030008CEA90E00E94AA021092BB051092BC0597
:103040001092BD051092BE051092BF051092C005EA
:103050001092C1050E944217AF9A8091BB05882348
:1030600009F055C08091BC05882309F050C08091BB
:10307000BF05813009F04BC09091C005913009F037
:1030800046C08091C105882309F041C09093BB05DB
:103090000E94A315AF9A88EE93E028EC30E0F90186
:1030A0003197F1F70197D9F70E944217AF9A8091B3
:1030B000BB058823D1F48091BC058823B1F48091AD
:1030C000BF05813091F48091C005813071F4809109
:1030D000C105882351F40E946E028AEB90E00E94A1
:1030E000AA0283E00E94D115FFCF0E946E0284ECF9
:1030F00090E00E94AA0286E00E94D11582E09DE045
:1031000028EC30E0F9013197F1F70197D9F70E94E7
:103110006E0283ED90E00E94AA020E94220480E5E4
:103120008DB9709A81E08093C2050E94F4068823CD
:10313000A9F01092C2050E946E028FED90E00E94ED
:10314000AA0286E00E94D11582E09DE028EC30E0E2
:10315000F9013197F1F70197D9F702C00E94580998
:103160000E946E02AF9808952F923F924F925F9205
:103170006F927F928F929F92AF92BF92CF92DF9287
:10318000EF92FF920F931F93DF93CF9300D0CDB7B1
:10319000DEB70E946E0280EF90E00E94AA0281E0FA
:1031A0000E94D115AE9A88EB9BE028EC30E0F90143
:1031B0003197F1F70197D9F70E946E020E944217EA
:1031C0008DB79EB70A970FB6F8949EBF0FBE8DBFFE
:1031D000EDB7FEB7319679E9E72E75E0F72EADB77A
:1031E000BEB71296FC92EE9211978FEF90E0938308
:1031F00082838091BD05848315828091BC0586837E
:1032000017828091BB05808711860E94FD20EDB753
:10321000FEB73A960FB6F894FEBF0FBEEDBF0E9400
:103220006E02C7010E94AA020E94E21611E0FA8211
:10323000E982E980FA8065E8B62E57E1C52E51E0B3
:10324000D52E4EE2842E41E0942E0E94B116082F16
:103250008823D9F385E00E94D115023021F0053092
:1032600009F072C004C0115009F461C003C01F5FAF
:10327000143040F4123069F1133009F459C01130A0
:1032800009F05CC08B2D8A95F1F78DB79EB70A9730
:103290000FB6F8949EBF0FBE8DBFEDB7FEB7319647
:1032A000ADB7BEB71196EC9211971296FC92D382ED
:1032B000C2828091BD05848315828091BC0586837E
:1032C00017828091BB05808711860E94FD2011E046
:1032D00025C08B2D8A95F1F78DB79EB70A970FB64B
:1032E000F8949EBF0FBE8DBFEDB7FEB73196ADB758
:1032F000BEB71196EC9211971296FC92938282823D
:103300008091BF05848315828091C00586831782D2
:103310008091C105808711860E94FD20EDB7FEB720
:103320003A960FB6F894FEBF0FBEEDBF07C013E08C
:1033300089E995E065E471E00E94F6200E946E0242
:1033400089E995E00E94AA020E94E216043009F081
:103350007CCF123009F42EC1133009F457C211305A
:1033600009F02CCF0E9442178091BB058093870300
:103370008091BC05809388038091BD05809389036B
:1033800011E039E9432E35E0532E24E6A22E21E048
:10339000B22E99E7892E91E0992E8FE4E82E81E0F4
:1033A000F82E08ECC02ED12CBBE37B2EA7E16A2EB1
:1033B0001230C9F0133059F1113009F051C08DB7F6
:1033C0009EB70A970FB6F8949EBF0FBE8DBFEDB79C
:1033D000FEB73196ADB7BEB712965C924E9211977A
:1033E000F382E28227C08DB79EB70A970FB6F89492
:1033F0009EBF0FBE8DBFEDB7FEB73196ADB7BEB75E
:1034000012965C924E921197B382A28213C08DB72E
:103410009EB70A970FB6F8949EBF0FBE8DBFEDB74B
:10342000FEB73196ADB7BEB712965C924E92119729
:10343000938282828091890384831582809188039C
:103440008683178280918703808711860E94FD20E2
:10345000EDB7FEB73A960FB6F894FEBF0FBEEDBFBC
:103460000E946E0289E995E00E94AA020E94B116AC
:10347000082F8823D9F3843031F0863021F085E09D
:103480000E94D11507C088E592E0F6013197F1F767
:103490000197D9F7013019F0033061F405C01150DC
:1034A00009F081C013E07FC01F5F143008F47BC0B7
:1034B00011E079C0023021F0053009F051C028C078
:1034C000123081F01330C9F0113009F06CC08091D6
:1034D00089038F5F80938903883108F464C0109258
:1034E000890361C0809188038F5F809388038C3348
:1034F00008F459C01092880356C0809187038F5FEB
:10350000809387038C3308F44EC0109287034BC01E
:10351000123081F01330C9F0113009F044C08091AD
:103520008903882319F4609289033DC081508093F8
:10353000890339C080918803882319F47092880325
:1035400032C08150809388032EC0809187038823E6
:1035500019F47092870327C081508093870323C09A
:103560000430A1F40E944217809187038093BB0529
:10357000809188038093BC05809189038093BD0569
:1035800085E00E94D1150E94F1160BC0063059F457
:103590000E946E028FE891E00E94AA0284E00E94DD
:1035A000D11501E001C000E00E94E216002309F4F9
:1035B000FFCE04CE0E9442178091C10580938703FD
:1035C0008091C005809388038091BF058093890313
:1035D00011E0F9E92F2EF5E03F2EEFEAAE2EE1E003
:1035E000BE2E75EC872E71E0972E69E9E62E61E01C
:1035F000F62E58ECC52ED12C772473944CE0642E13
:1036000033E6532E2FE1422E1230C9F0133059F118
:10361000113009F051C08DB79EB70A970FB6F894D4
:103620009EBF0FBE8DBFEDB7FEB73196ADB7BEB72B
:1036300012963C922E921197F382E28227C08DB7A8
:103640009EB70A970FB6F8949EBF0FBE8DBFEDB719
:10365000FEB73196ADB7BEB712963C922E92119737
:10366000B382A28213C08DB79EB70A970FB6F894A3
:103670009EBF0FBE8DBFEDB7FEB73196ADB7BEB7DB
:1036800012963C922E9211979382828280918903A6
:1036900084831582809188038683178280918703B3
:1036A000808711860E94FD20EDB7FEB73A960FB6CF
:1036B000F894FEBF0FBEEDBF0E946E0289E995E04F
:1036C0000E94AA020E94B116082F8823D9F38430E1
:1036D00031F0863021F085E00E94D11507C088E5E1
:1036E00092E0F6013197F1F70197D9F7013019F01F
:1036F000033061F405C0115009F081C013E07FC0B0
:103700001F5F143008F47BC011E079C0023021F053
:10371000053009F051C028C0123081F01330C9F0D3
:10372000113009F06CC0809189038F5F8093890309
:10373000803208F464C01093890361C080918803CB
:103740008F5F809388038D3008F459C0709288038E
:1037500056C0809187038F5F80938703843608F477
:103760004EC0109287034BC0123081F01330C9F065
:10377000113009F044C080918903813019F44092DE
:1037800089033DC081508093890339C080918803AB
:10379000813019F46092880332C08150809388038D
:1037A0002EC080918703882319F45092870327C085
:1037B00081508093870323C00430A1F40E944217F4
:1037C000809187038093C105809188038093C00511
:1037D000809189038093BF0585E00E94D1150E94E6
:1037E000F1160BC0063059F40E946E028FE891E08A
:1037F0000E94AA0284E00E94D11501E001C000E00D
:103800000E94E216002309F4FFCED8CCAF980E94A4
:10381000E216AE980F900F90CF91DF911F910F910C
:10382000FF90EF90DF90CF90BF90AF909F908F90E0
:103830007F906F905F904F903F902F900895CF9220
:10384000DF92EF92FF920F931F93CF93DF93AF9A84
:103850008E9A88EE93E00197F1F78E9880E58A952D
:10386000F1F780B38CEA93E00197F1F7869B91C062
:103870008CEC0E94960384E40E949603AF988CE43B
:103880009DE128EC30E0F9013197F1F70197D9F784
:10389000AF9A8E9AF8EEEF2EF3E0FF2EC701019754
:1038A000F1F78E98E0E5DE2E8D2D8A95F1F780B345
:1038B0000CEA13E0C8010197F1F780B38CEC0E9489
:1038C00096038EEB0E9496030E94B703C82E0E94B7
:1038D000B703282F8E9AC7010197F1F78E98DA94D3
:1038E000F1F780B3C8010197F1F780B3722F60E060
:1038F0006C0D711D882777FD8095982F0E94DB1E27
:1039000020E030E040E85DE30E94E11D41E021E07D
:1039100007E813E00E94D520AF98A2E5B3E01D921E
:1039200083E0A636B807D9F7CDB7DEB72C970FB628
:10393000F894DEBF0FBECDBFEDB7FEB731965497FA
:10394000BA83A9838CED91E0938382838091BD0536
:10395000848315828091BC05868317828091BB0584
:103960008087118687E893E0938782870E94FD20F5
:103970008DB79EB70C960FB6F8949EBF0FBE8DBF45
:10398000DF91CF911F910F91FF90EF90DF90CF903B
:10399000089587E893E060EF71E00E94F620BCCFC5
:1039A0004F925F926F927F928F929F92AF92BF924F
:1039B000CF92DF92EF92FF921F93CF93DF930E94FB
:1039C0000C1780ED97E028EC30E0F9013197F1F722
:1039D0000197D9F70E946E0284EF91E00E94AA023B
:1039E00080E49FE128EC30E0F9013197F1F701978D
:1039F000D9F70E946E0285E092E00E94AA0280E45C
:103A00009FE128EC30E0F9013197F1F70197D9F700
:103A10000E9415180E94B116049711F40E94B41860
:103A20000E946E0285E192E00E94AA0282E00E945A
:103A3000D11513E6C0E0D0E039E9C32E35E0D32E2E
:103A40002EE2422E22E0522E9DE1692E92E0792E46
:103A500087E8882E83E0982EBFEDAB2EB12CA8EC22
:103A6000EA2EF12C0E9442170E941F1C8091C20571
:103A7000813009F0AF9AC130D10561F1C230D10572
:103A800009F458C0209709F05BC08DB79EB70C971A
:103A90000FB6F8949EBF0FBE8DBFEDB7FEB731963F
:103AA000ADB7BEB71296DC92CE9211977382628246
:103AB0008091BD05848315828091BC058683178221
:103AC00091868086B386A2860E94FD208DB79EB720
:103AD0000C962AC0ADB7BEB71E970FB6F894BEBFFE
:103AE0000FBEADBFEDB7FEB731961296DC92CE9207
:103AF0001197538242828091BD0584831582809103
:103B0000BC05868317828091BF05808711868091CE
:103B1000C005828713868091C105848715860E941F
:103B2000FD208DB79EB70E960FB6F8949EBF0FBEC0
:103B30008DBF06C089E995E06FED70E00E94F62028
:103B40000E946E0289E995E00E94AA02AE9A8CED6D
:103B500095E0F7013197F1F70197D9F7AE98809189
:103B6000C205813099F48091BC05181779F088233B
:103B700029F065E00E94F725992331F4AF9A8CE68D
:103B800093E00E94C911AF981091BC0588E199E7B4
:103B9000F7013197F1F70197D9F721968091C20586
:103BA000813041F480E090E0219711F481E090E0D1
:103BB000EC0158CFC330D1050CF454CFC0E0D0E0B5
:103BC00051CFA0E2B0E0E7EEFDE10C942526698339
:103BD0007A838B839C832D833E834F835887CE01CA
:103BE0000196BE01675F7F4F0E945D20CE01059662
:103BF000BE016F5E7F4F0E945D209985923088F0F4
:103C000089898230C8F0943019F4823051F404C0AC
:103C1000843029F4923081F489E492E0C6C0923075
:103C200049F420E09A858A89981321E02A87CE01F9
:103C30000996BBC0823049F420E09A858A8998139E
:103C400021E02A8BCE014196B0C02D843E844F8462
:103C500058886D887E888F88988CEE24FF24870191
:103C6000AA24BB24650140E050E060E070E0E0E0A1
:103C7000F0E0C10181709070892BE9F0E60CF71C2F
:103C8000081D191D9A01AB012A0D3B1D4C1D5D1D20
:103C900080E090E0A0E0B0E0E614F7040805190524
:103CA00020F481E090E0A0E0B0E0BA01A901480F63
:103CB000591F6A1F7B1FAA0CBB1CCC1CDD1C97FE66
:103CC00008C081E090E0A0E0B0E0A82AB92ACA2AA2
:103CD000DB2A3196E032F10549F0660C771C881C2E
:103CE000991C5694479437942794C3CFFA85EA8950
:103CF0002B893C898B859C85280F391F2E5F3F4F70
:103D000017C0CA0181709070892B61F016950795D4
:103D1000F794E79480E090E0A0E0B0E8E82AF92A80
:103D20000A2B1B2B76956795579547952F5F3F4F2D
:103D300077FDE7CF0CC0440F551F661F771F17FD97
:103D40004160EE0CFF1C001F111F2150304040301D
:103D500090E0590790E0690790E4790760F32B8FB2
:103D60003C8FDB01CA018F779070A070B0708034F7
:103D70009105A105B10561F447FD0AC0E114F10404
:103D80000105110529F0405C5F4F6F4F7F4F407870
:103D90001A8EFE1711F081E08A8F4D8F5E8F6F8F24
:103DA00078A383E0898FCE0149960E94881FA09650
:103DB000E2E10C944126A8E0B0E0E1EEFEE10C94D3
:103DC0002E269B01AC0183E08983DA01C901882793
:103DD000B7FD83959927AA27BB27B82E2115310552
:103DE0004105510519F482E089833AC08823A9F07E
:103DF000203080E0380780E0480780E8580729F441
:103E000060E070E080E09FEC30C0EE24FF2487018A
:103E1000E21AF30A040B150B02C079018A018EE144
:103E2000C82ED12CDC82CB82ED82FE820F831887D4
:103E3000C801B7010E94391F01971816190684F4AA
:103E4000082E04C0EE0CFF1C001F111F0A94D2F7AD
:103E5000ED82FE820F831887C81AD90ADC82CB82D2
:103E6000BA82CE0101960E94881F2896E9E00C9440
:103E70004A26EF92FF920F931F937B018C0180E003
:103E8000E81680E0F80681E0080780E0180788F46B
:103E90008FEFE816F1040105110531F028F088E0F4
:103EA00090E0A0E0B0E017C080E090E0A0E0B0E0DB
:103EB00012C080E0E81680E0F80680E0080781E0A4
:103EC000180728F088E190E0A0E0B0E004C080E1AD
:103ED00090E0A0E0B0E020E230E040E050E0281BBD
:103EE000390B4A0B5B0B04C016950795F794E794C2
:103EF0008A95D2F7F701EF5AFD4F8081281B3109CF
:103F000041095109C9011F910F91FF90EF90089548
:103F1000DF92EF92FF920F931F93FC01E480F580F4
:103F200006811781D1808081823048F480E090E062
:103F3000A0E1B0E0E82AF92A0A2B1B2BA5C08430A7
:103F400009F49FC0823021F4EE24FF24870105C0CC
:103F5000E114F1040105110519F4E0E0F0E096C068
:103F6000628173819FEF623879070CF05BC022E8B1
:103F70003FEF261B370B2A3131052CF020E030E0D3
:103F800040E050E02AC0B801A701022E04C0769597
:103F90006795579547950A94D2F781E090E0A0E0A5
:103FA000B0E004C0880F991FAA1FBB1F2A95D2F743
:103FB0000197A109B1098E219F21A023B123009768
:103FC000A105B10521F081E090E0A0E0B0E09A0108
:103FD000AB01282B392B4A2B5B2BDA01C9018F77D8
:103FE0009070A070B07080349105A105B10539F4CE
:103FF00027FF09C0205C3F4F4F4F5F4F04C0215C3B
:104000003F4F4F4F5F4FE0E0F0E02030A0E03A0735
:10401000A0E04A07A0E45A0710F0E1E0F0E07901DF
:104020008A0127C06038710564F5FB01E158FF4F34
:10403000D801C7018F779070A070B070803491055F
:10404000A105B10539F4E7FE0DC080E490E0A0E0E1
:10405000B0E004C08FE390E0A0E0B0E0E80EF91E0D
:104060000A1F1B1F17FF05C016950795F794E794C5
:10407000319687E016950795F794E7948A95D1F7DE
:1040800005C0EE24FF248701EFEFF0E06E2F679567
:1040900066276795902F9F77D794DD24D7948E2F2E
:1040A0008695492F462B582F5D29B701CA011F91CC
:1040B0000F91FF90EF90DF900895FC01DB014081AC
:1040C00051812281622F6F7770E0221F2227221FE9
:1040D0009381892F880F822B282F30E0991F9927F1
:1040E000991F11969C93119721153105A9F541153A
:1040F00051056105710511F482E037C082E89FEF38
:1041000013969C938E9312979A01AB0167E0220F4E
:10411000331F441F551F6A95D1F783E08C930DC060
:10412000220F331F441F551F12968D919C91139798
:10413000019713969C938E931297203080E0380756
:1041400080E0480780E4580758F314962D933D9378
:104150004D935C93179708952F3F310579F44115DE
:1041600051056105710519F484E08C93089564FF8D
:1041700003C081E08C9312C01C9210C02F573040B6
:1041800013963C932E93129783E08C9387E0440F11
:10419000551F661F771F8A95D1F7706414964D934B
:1041A0005D936D937C9317970895EF92FF920F9311
:1041B0001F93F22FF02E47FD02C0E4E001C0E4E1BE
:1041C000242F332727FD309537FF03C030952195E5
:1041D0003F4F4F2D512F0F2FEE2E0E94FE228F2D7D
:1041E000912F1F910F91FF90EF900895FB01DC013B
:1041F00001900D920020E1F70895AEE0B0E0E3E019
:10420000F1E20C9433260D891E8986E08C831A8393
:1042100009838FEF9FE79E838D839E01275E3F4F2B
:10422000CE0101966F89788DA9010E9421212F81ED
:104230003885020F131FF80110822E96E4E00C94CB
:104240004F26ABE0B0E0E7E2F1E20C9425263C011A
:104250002B015A01FC0117821682838181FD03C064
:104260006FEF7FEFC6C19AE0892E1E010894211CD2
:10427000311CF3012381F20123FD859123FF8191FC
:104280002F01882309F4B2C1853239F423FD8591C9
:1042900023FF81912F01853229F490E0B3010E9420
:1042A0004E25E7CF982FFF24EE249924FFE1FF1538
:1042B000D0F09B3269F09C3228F4903259F093325E
:1042C00091F40EC09D3249F0903369F441E024C06E
:1042D00052E0F52A84E0F82A28C098E0F92A25C09F
:1042E000E0E1FE2A22C0F7FC29C0892F80538A30E2
:1042F00070F4F6FE05C0989C902C1124980E15C001
:10430000E89CE02C1124E80EF0E2FF2A0EC09E3259
:1043100029F4F6FC6BC140E4F42A07C09C3619F47A
:1043200050E8F52A02C0983649F4F20123FD959130
:1043300023FF91912F01992309F0B8CF892F85543C
:10434000833018F08052833038F444E050E0A40EFB
:10435000B51E5FE359830FC0933631F0933779F080
:10436000933509F056C020C0F5018081898342E071
:1043700050E0A40EB51E610101E010E012C0F5018D
:10438000C080D180F6FC03C06FEF7FEF02C0692DC3
:1043900070E042E050E0A40EB51EC6010E94432525
:1043A0008C015FE7F52214C0F501C080D180F6FCD6
:1043B00003C06FEF7FEF02C0692D70E042E050E074
:1043C000A40EB51EC6010E9438258C0150E8F52ABE
:1043D000F3FE07C01AC080E290E0B3010E944E25B0
:1043E000EA948E2D90E008171907A8F30EC0F60185
:1043F000F7FC8591F7FE81916F0190E0B3010E9477
:104400004E25E110EA94015010400115110579F78D
:10441000EAC0943611F0993669F5F7FE08C0F50147
:10442000208131814281538184E090E00AC0F5010E
:10443000808191819C01442737FD4095542F82E073
:1044400090E0A80EB91E9FE6F92257FF09C05095CB
:104450004095309521953F4F4F4F5F4FE0E8FE2A42
:10446000CA01B901A1012AE030E00E947A25D82EC4
:10447000D21840C0953729F41F2D1F7E2AE030E066
:104480001DC01F2D197F9F3661F0903720F498359D
:1044900009F0ACC00FC0903739F0983709F0A6C0CA
:1044A00004C028E030E00AC0106114FD146020E16F
:1044B00030E004C014FD166020E132E017FF08C0B0
:1044C000F501608171818281938144E050E008C0F0
:1044D000F50180819181BC0180E090E042E050E0F4
:1044E000A40EB51EA1010E947A25D82ED2188FE7FE
:1044F000F82EF122F6FE0BC05EEFF522D91438F447
:10450000F4FE07C0F2FC05C08FEEF82202C01D2D9C
:1045100001C0192DF4FE0DC0FE01ED0DF11D8081CD
:10452000803319F499EEF92208C01F5FF2FE05C02E
:1045300003C08F2D867809F01F5F0F2DF3FC14C088
:10454000F0FE0FC01E1510F09D2C0BC09D2C9E0C74
:10455000911A1E2D06C080E290E0B3010E944E2504
:104560001F5F1E15C0F304C01E1510F4E11A01C030
:10457000EE2404FF0FC080E390E0B3010E944E25BB
:1045800002FF1DC001FD03C088E790E00EC088E572
:1045900090E00BC0802F867891F001FF02C08BE283
:1045A00001C080E2F7FC8DE290E0B3010E944E254D
:1045B00006C080E390E0B3010E944E259A94D9147E
:1045C000C0F3DA94F101ED0DF11D808190E0B301AB
:1045D0000E944E25DD20A9F706C080E290E0B301DD
:1045E0000E944E25EA94EE20C1F743CEF301668186
:1045F0007781CB012B96E2E10C944126A9E0B0E053
:10460000E4E0F3E20C9429266A01122FA02EBE2CBE
:104610002BE3201718F42CE3922E02C0902E9394D3
:10462000AE014F5F5F4F27E0092D0E946024BC015F
:104630008981E82EFF24C70189709070019711F4D9
:10464000ADE209C0B1FE02C0ABE205C0B0FC02C0E1
:10465000A0E001C0A0E2E3FE3BC0AA2311F423E0E6
:1046600001C024E0211710F020E002C0121B212F0E
:10467000EB2CB4FE02C0322F0AC0F601322F80E2CA
:1046800002C0819331503323E1F7C20ED11CAA231B
:1046900019F0F601A1936F01F6013196E2FE05C013
:1046A0009EE4D6019C9381E404C09EE6D6019C93CF
:1046B00081E611968C9391833296DF01832F90E2ED
:1046C00002C09D9381508823E1F7E30FF11D40C0A4
:1046D000E2FE42C0AA2311F423E001C024E0211726
:1046E00010F020E002C0121B212FEB2CB4FE02C000
:1046F000922F0AC0F601922F80E202C0819391505E
:104700009923E1F7C20ED11CAA2319F0F601A19357
:104710006F01F6013196E2FE08C089E4D6018C9360
:104720008EE411968C9386E407C089E6D6018C93BB
:104730008EE611968C9386E681833296DF01892F6F
:1047400020E202C02D9381508823E1F7E90FF11D8B
:1047500010822EEF3FEFAFC0161617061CF041E097
:1047600050E003C0AB014F5F5F4FAA2019F480E017
:1047700090E003C08A2D90E0019620E030E0AA236B
:1047800011F021E030E0240F351F280F391F812F51
:1047900090E02817390714F020E002C0121B212FE7
:1047A0004B2D50E0CA0180719070B4FC0DC0B3FC79
:1047B0000BC0F601322F40E202C041933150332347
:1047C000E1F7C20ED11C01C0322FAA2319F0F60165
:1047D000A1936F01892B11F0132F0AC0F601132F3B
:1047E00080E302C0819311501123E1F7C30ED11C65
:1047F000092D060FBA8090E1892E912C8E209F20E2
:10480000E4FE04C0F1E3BF1609F40150101614F0E1
:1048100001E003C0093008F008E09B0177FF02C007
:1048200020E030E0CB010196821B930BFE01319614
:10483000E80FF91F8EE2F82E3B01601A71088A2DED
:1048400090E044275527481B590B8FEF2F3F38071F
:1048500019F4D601FD926D01621773072CF06216F0
:10486000730614F4808101C080E3215030403196FA
:104870002417350724F0D6018D936D01E6CF261756
:10488000370749F4B5E3BB1528F0BB1621F48114B2
:10489000910409F481E3F6018193D601812F90E21E
:1048A00002C09C93815011968823D9F7E10FF11D26
:1048B000108220E030E0C9012996EEE00C944526F4
:1048C000283008F027E03327DA01990F311D87FDE2
:1048D000916000966105710539F432602E5F3D9359
:1048E00030E32A95E1F708959F3F30F08038710555
:1048F000610509F03C5F3C5F3D93913008F08068B2
:10490000911DDF93CF931F930F93FF92EF92192F77
:10491000987F9695E92F96959695E90FFF27E05198
:10492000FD4F99273327EE24FF24A701E7010590C7
:104930000894079428F4360FE71EF81E491F511DEE
:10494000660F771F881F991F0694A1F7059007949B
:1049500028F4E70EF81E491F561FC11D770F881F48
:10496000991F661F0694A1F70590079428F4F80E86
:10497000491F561FC71FD11D880F991F661F771F1C
:104980000694A1F70590079420F4490F561FC71FFE
:10499000D81F990F661F771F881F0694A9F7849167
:1049A0001095177041F0D695C79557954795F79490
:1049B000E7941A95C1F7E6E9F2E06894159015912D
:1049C00035916591959105907FE27395E118F10A13
:1049D000430B560BC90BD009C0F7E10CF11E431F66
:1049E000561FC91FD01D7EF4703311F48A95E6CF8F
:1049F000E894015030F0080F0AF40027021708F479
:104A0000202F2395022F7A3328F079E37D932A957E
:104A1000E9F710C07D932A9589F6069497956795D6
:104A2000379517951794E118F10A430B560BC90BEC
:104A3000D00998F023957E9173957A3308F070E34E
:104A40007C932013B8F77E9170617D9330F083954D
:104A500071E37D9370E32A95E1F71124EF90FF90C5
:104A60000F911F91CF91DF91992787FD9095089520
:104A7000FC010590615070400110D8F78095909529
:104A80008E0F9F1F0895FC0161507040019001102E
:104A9000D8F7809590958E0F9F1F08950F931F93C1
:104AA000CF93DF938C01EB018B8181FF1BC082FFD1
:104AB0000DC02E813F818C819D812817390764F4B8
:104AC000E881F9810193F983E88306C0E885F985D7
:104AD000802F0995892B31F48E819F8101969F83C8
:104AE0008E8302C00FEF1FEFC801DF91CF911F919E
:104AF0000F910895FA01AA27283051F1203181F150
:104B0000E8946F936E7F6E5F7F4F8F4F9F4FAF4FD5
:104B1000B1E03ED0B4E03CD0670F781F891F9A1FE8
:104B2000A11D680F791F8A1F911DA11D6A0F711D9C
:104B3000811D911DA11D20D009F468943F912AE0A8
:104B4000269F11243019305D3193DEF6CF01089590
:104B5000462F4770405D4193B3E00FD0C9F7F6CFC1
:104B6000462F4F70405D4A3318F0495D31FD405289
:104B7000419302D0A9F7EACFB4E0A695979587951F
:104B800077956795BA95C9F70097610571050895FE
:104B90009B01AC010A2E06945795479537952795AA
:104BA000BA95C9F7620F731F841F951FA01D089542
:104BB000629FD001739FF001829FE00DF11D649F01
:104BC000E00DF11D929FF00D839FF00D749FF00D8D
:104BD000659FF00D9927729FB00DE11DF91F639F2E
:104BE000B00DE11DF91FBD01CF0111240895991BDE
:104BF00079E004C0991F961708F0961B881F7A95D4
:104C0000C9F780950895A1E21A2EAA1BBB1BFD01CE
:104C10000DC0AA1FBB1FEE1FFF1FA217B307E4079B
:104C2000F50720F0A21BB30BE40BF50B661F771FF3
:104C3000881F991F1A9469F76095709580959095D3
:104C40009B01AC01BD01CF0108952F923F924F927D
:104C50005F926F927F928F929F92AF92BF92CF920C
:104C6000DF92EF92FF920F931F93CF93DF93CDB715
:104C7000DEB7CA1BDB0B0FB6F894DEBF0FBECDBF8D
:104C800009942A88398848885F846E847D848C845E
:104C90009B84AA84B984C884DF80EE80FD800C8167
:104CA0001B81AA81B981CE0FD11D0FB6F894DEBF4A
:0C4CB0000FBECDBFED010895F894FFCFBA
:104CBC0030782020202020202020002020202020A0
:104CCC0020202020202020204279746573005A6116
:104CDC007069737977616E69652E2E2E005A616B3F
:104CEC006F6E637A6F6E6F2E00253032642D253017
:104CFC0032642D253032642E7478740053454C4642
:104D0C00544553543A2052544300426C616420522F
:104D1C005443210020205573746177207A656761B4
:104D2C0072210053454C46544553543A5344004267
:104D3C0072616B205344207A204641543332210057
:104D4C0020204B4F4E464947555241434A41003172
:104D5C003E435A41533A20253032643A253032646E
:104D6C003A253032640A00313E435A41533A2025E9
:104D7C003032643A253032643A2530326400323EA7
:104D8C00444154413A20253032642D253032642D73
:104D9C002530326400333E5A414B4F4E435A00206B
:104DAC005B253032645D3A2025303264203A202570
:104DBC0030326400202025303264203A5B253032BA
:104DCC00645D3A2025303264002020253032642086
:104DDC003A2025303264203A5B253032645D004144
:104DEC006E756C6F77616E6F005B253032645D2D74
:104DFC002025303264202D203230253032640020C2
:104E0C0025303264202D5B253032645D2D2032300C
:104E1C0025303264002025303264202D202530329C
:104E2C0064202D5B3230253032645D0025303264D5
:104E3C003A253032643A253032643B25730D0A0032
:104E4C00455252002D2D2D54656D704C6F67676562
:104E5C00722D2D2D00204669726D7761726520765A
:104E6C00302E323000476F746F77792E0025303238
:104E7C00643A25303264202538732563430025308D
:104E8C0032643A2530326420253032642D2530329C
:104E9C00642D323025303264000000000000000028
:104EAC0000000102020303030304040404040404C9
:104EBC000405050505050505050505050505050597
:104ECC000506060606060606060606060606060677
:104EDC000606060606060606060606060606060666
:104EEC000607070707070707070707070707070747
:104EFC000707070707070707070707070707070736
:104F0C000707070707070707070707070707070725
:104F1C000707070707070707070707070707070715
:104F2C0007080808080808080808080808080808F6
:104F3C0008080808080808080808080808080808E5
:104F4C0008080808080808080808080808080808D5
:104F5C0008080808080808080808080808080808C5
:104F6C0008080808080808080808080808080808B5
:104F7C0008080808080808080808080808080808A5
:104F8C000808080808080808080808080808080895
:104F9C000808080808080808080808080808080885
:024FAC000800FB
:00000001FF
